:020000020000FC
:1000000019C018E01A95F1F708950AE030950894A0
:1000100010F4D99A02C0D9980000F3DFF2DF3695C8
:100020000A95B1F708951FEF2AE02A95F1F71A957E
:10003000D9F7089510E820E016BD26BD11E01EBFD7
:100040001FE51DBF3F9A3E983C9A3D9A3C9A3B9AC9
:100050003A983998389AD798D398379A35983398E8
:10006000329A31983098BA9AC29813E310BF11E0CF
:1000700013BFD99AD19A31E0C8DFD5DF32E0C5DFAE
:10008000D2DF33E0C2DFCFDF34E0BFDFCCDF48ECCC
:10009000369A3699FECF50910500352FB6DF30E005
:0A00A000B4DF5CBF4A95A1F7E6CF7C
:00000001FF
